:100000000C94BF000C9416010C9427010C94DC0096
:100010000C94DC000C94DC000C94DC000C940301C8
:100020000C94DC000C94DC000C94DC000C94DC00E0
:100030000C94DC000C948D010C94DC000C94DC001E
:100040000C94DC000C94DC000C94DC000C94DC00C0
:100050000C9438010C94DC000C9461010C94DC00CD
:100060000C9483010C94DC000C94DC000C94DC00F8
:100070000C94DC000C94DC000C94DC006E616E00CF
:10008000696E660000407A10F35A00A0724E18099B
:100090000010A5D4E80000E87648170000E40B54EF
:1000A000020000CA9A3B000000E1F50500008096BE
:1000B0009800000040420F000000A08601000000F0
:1000C000102700000000E8030000000064000000AA
:1000D00000000A00000000000100000000002C7673
:1000E000D888DC674F0823DFC1DFAE59E1B1B7968E
:1000F000E5E3E453C63AE651997696E8E6C28426EB
:10010000EB898C9B62ED407C6FFCEFBC9C9F40F2C6
:10011000BAA56FA5F490055A2AF75C936B6CF96742
:100120006DC11BFCE0E40D47FEF520E6B500D0ED07
:10013000902E0300943577050080841E080000206F
:100140004E0A000000C80C333333330F986E12830D
:100150001141EF8D2114893BE65516CFFEE6DB18E1
:10016000D1844B381BF77C1D901DA4BBE4242032A6
:1001700084725E228100C9F124ECA1E53D2711249F
:100180001FBECFEFD0E1DEBFCDBF11E0A0E0B1E0F8
:10019000E4EFF8E102C005900D92A434B107D9F75D
:1001A00021E0A4E4B1E001C01D92AA3DB207E1F74D
:1001B0000E94D5020C94780C0C940000F894909155
:1001C000C00095FF03C08093C60014C09091CB017E
:1001D000292F30E04091CA01241B31092038310514
:1001E00049F0E92FEF77F0E0E65BFE4F80839F5FF9
:1001F0009093CB01789480E090E008950E947D0474
:1002000080E090E008951F920F920FB60F92112494
:100210008F9389B182958F70806F8095809349010B
:100220008F910F900FBE0F901F9018951F920F92F5
:100230000FB60F9211248F93469A429881E08093D3
:1002400045018F910F900FBE0F901F9018951F9230
:100250000F920FB60F9211248F93479A439881E023
:10026000809346018F910F900FBE0F901F901895AD
:100270001F920F920FB60F9211248F93EF93FF935B
:100280008091C6008093480180914701811104C08C
:1002900080914801853569F4E0914701F0E0809153
:1002A0004801E453FE4F8083809147018F5F809324
:1002B0004701FF91EF918F910F900FBE0F901F900C
:1002C00018951F920F920FB60F9211248F93EF93F0
:1002D000FF93E091CA018091CB01E81761F0EF77BD
:1002E000F0E0E65BFE4F80818093C600EAECF1E02F
:1002F00080818F5F8083FF91EF918F910F900FBE70
:100300000F901F9018951F920F920FB60F92112405
:100310000F900FBE0F901F9018951F920F920FB65F
:100320000F9211248F9381E0809344018F910F905D
:100330000FBE0F901F90189584B7877F84BFE0E6AB
:10034000F0E08081886180831082E9E6F0E08081BE
:100350008A6080838DB383608DBB88B1806C88B9DF
:1003600087B18C6C87B9599A519A1092C50086E270
:100370008093C40022E02093C00088ED8093C100E8
:1003800086E08093C20084B1876B84B985B1806BAD
:1003900085B980E58CBD84E08093B8008093BC0073
:1003A0008DE08093810080E094E0909389008093B9
:1003B000880020936F00ECE7F0E08081806C808300
:1003C00084E880937A008FEF80937E0088E08093AA
:1003D000680080EF809373007894089595B16770FA
:1003E000987F692B65B92C9891E19EBD0DB407FEED
:1003F000FDCF8EBD0DB407FEFDCF2C9A0895CF9290
:10040000DF92EF92FF92CF936A017B01C82FC170F8
:100410002BE734E14EEC51E4C701B6010E9484069B
:100420000E94CA05F62E64E06C0F8F2D0E94EE012B
:100430006F2D70E080E090E00E94F6052BE734E13C
:100440004EEC51E40E946205CF91FF90EF90DF9057
:10045000CF900895CF92DF92EF92FF92CF936A01EF
:100460007B018170C82FCC0F22E03BE247E051E4D2
:10047000C701B6010E94840622E73AE84EE051E443
:100480000E94FD040E94CA05F62E61E06C0F8F2DBC
:100490000E94EE016F2D70E080E090E00E94F60572
:1004A00022E73AE84EE051E40E94FE0422E03BE2FB
:1004B00047E051E40E946205CF91FF90EF90DF90FA
:1004C000CF900895CF92DF92EF92FF92CF936A017F
:1004D0007B01C82FC17020E030E04FE753E4C70133
:1004E000B6010E94840625E33EE542E050E40E9406
:1004F00062050E94CA05F62E6C2F660F8F2D0E9492
:10050000EE016F2D70E080E090E00E94F60525E39B
:100510003EE542E050E40E94840620E030E04FE7F0
:1005200053E40E946205CF91FF90EF90DF90CF904F
:100530000895CF92DF92EF92FF920F931F93CF9384
:10054000DF93EC016A017B01C901B801A7019601A3
:100550000E94FD049B01AC0163E373E383E590E437
:100560000E946205AB01BC0188810E942A02698356
:100570007A838B839C832AE43CE042E45FE3C701F7
:10058000B6010E948406AB01BC0188810E94620210
:100590006D837E838F839887DF91CF911F910F9119
:1005A000FF90EF90DF90CF900895CF93DF93CDB77A
:1005B000DEB76A970FB6F894DEBF0FBECDBF1982C3
:1005C0001A861B861C861D8681E08E871F8A188EE0
:1005D000198E1A8E8EE091E09093D7018093D60108
:1005E0000E949C010E94CD048CE191E00E94ED0BE1
:1005F00020E031E040E150E061E070E083E291E032
:100600000E94B90B61E080E00E94C30420E031E069
:1006100040E150E061E070E083E291E00E94B90BBC
:1006200040E050E0BA0180E00E94FF0140E050E06D
:10063000BA0181E00E94FF010AE919E929E13FE3DB
:1006400043E353E363EB7EE3CE0101960E949902FC
:1006500000E010E020E830E440E050E060E87FE3B4
:10066000CE010E960E949902C12CD12C0F2EF5E4DA
:10067000EF2EF1E0FF2EF02D06E411E00F2EFDEC41
:10068000AF2EF1E0BF2EF02D0F2EF3ED2F2EF1E067
:100690003F2EF02D0F2EFCE74F2E512CF02D0F2E5C
:1006A000FAE76F2E712CF02D0F2EF8E78F2E912C7C
:1006B000F02DF70180818130B1F460E080E00E948C
:1006C000C30420E031E04FE050E061E070E084E3FB
:1006D00091E00E94B90BF70110828FE295E7019734
:1006E000F1F700C00000F80180818130B1F461E0D1
:1006F00080E00E94C30420E031E04FE050E061E080
:1007000070E084E391E00E94B90BF80110828FE25F
:1007100095E70197F1F700C0000080914701823012
:1007200059F4F5018081823539F4F894E0E6F0E07F
:10073000808188618083FFCF809147018830A9F450
:1007400010924701F5018081EEECF1E08081EFEC41
:10075000F1E08081E0EDF1E08081E1EDF1E0808188
:10076000E2EDF1E08081F1018081809144018823F4
:10077000E9F110924401CC2061F1F4018081E9E7B4
:10078000F0E08081F1E0DF1671F0DF1638F082E0F2
:10079000D81671F093E0D91681F014C060E080E0C3
:1007A0000E94C30481C061E080E00E94C3047CC059
:1007B00060E089E00E94C30477C061E089E00E94A4
:1007C000C30404C0D394E4E0DE120FC0C12CD12CCA
:1007D0000DC0F2018081887F8D298083F3018081A3
:1007E00080648083CC24C39401C0C12C80914901D2
:1007F000823021F118F4813031F05BCF843041F147
:100800008830E1F156CF98B180E4892788B998B152
:1008100084E0892788B9469B07C040E050E0BA01D0
:1008200080E00E94FF0107C04A855B856C857D855D
:1008300080E00E94FF01109249013BCF88B18058AF
:1008400088B998B188E0892788B91092490131CFD9
:1008500020E030E040E05FE36A857B858C859D8504
:100860000E94FD04AB01BC014A875B876C877D87D2
:1008700080E00E94FF01109249011BCF20E030E090
:1008800040E05FE36A857B858C859D850E94FE0440
:10089000AB01BC014A875B876C877D8780E00E9443
:1008A000FF011092490105CFD394C12C9FCFECEBEF
:1008B000F0E09081906A908390819923ECF79EE418
:1008C0009093BB00ECEBF0E090819F7D9083908152
:1008D0009068908390819923ECF78093BB00ECEBB8
:1008E000F0E080818068808380818823ECF7ECEBE6
:1008F000F0E08081806980830895CF93DF93C82FD3
:10090000D82FD07F8D2F85600E9457048D2F816056
:100910000E94570480E1C89FE00111248C2F85605C
:100920000E9457048C2F81600E94570480E18A95B1
:10093000F1F7DF91CF910895CF93DF93C82FD82F90
:10094000D07F8D2F84600E9457048D2F0E94570402
:1009500020E1C29FC001112484600E9457048C2FA3
:100960008295807F0E945704C13039F48FE496E469
:100970000197F1F700C0000003C098E29A95F1F7E3
:10098000DF91CF91089561708F7090E4699F800D21
:10099000112480680E949C040895CF9380E00E94F7
:1009A00057042FEB84ED91E0215080409040E1F717
:1009B00000C00000C5E084E00E94570480E00E946F
:1009C0005704C150C1F728EC2A95F1F784E20E9440
:1009D000570480E20E9457048AE20E949C0488E047
:1009E0000E949C0481E00E949C0486E00E949C047A
:1009F0008CE00E949C04CF9108955058BB27AA27F1
:100A00000ED048C139D130F03ED120F031F49F3FB3
:100A100011F41EF42EC10EF4E095E7FB24C1E92F7A
:100A20004AD180F3BA17620773078407950718F055
:100A300071F49EF562C10EF4E0950B2EBA2FA02D35
:100A40000B01B90190010C01CA01A0011124FF277B
:100A5000591B99F0593F50F4503E68F11A16F04076
:100A6000A22F232F342F4427585FF3CF4695379575
:100A70002795A795F0405395C9F77EF41F16BA0B3A
:100A8000620B730B840BBAF09150A1F0FF0FBB1FE8
:100A9000661F771F881FC2F70EC0BA0F621F731F31
:100AA000841F48F4879577956795B795F7959E3F8E
:100AB00008F0B3CF9395880F08F09927EE0F97951C
:100AC000879508950CD0E6C0DED040F0D5D030F048
:100AD00021F45F3F19F0C7C0511110C1CAC0EBD05B
:100AE00098F39923C9F35523B1F3951B550BBB27F5
:100AF000AA2762177307840738F09F5F5F4F220FA2
:100B0000331F441FAA1FA9F333D00E2E3AF0E0E89A
:100B100030D091505040E695001CCAF729D0FE2FE6
:100B200027D0660F771F881FBB1F26173707480778
:100B3000AB07B0E809F0BB0B802DBF01FF2793582E
:100B40005F4F2AF09E3F510568F08DC0D7C05F3FD0
:100B5000ECF3983EDCF3869577956795B795F79516
:100B60009F5FC9F7880F911D9695879597F908950E
:100B7000E1E0660F771F881FBB1F621773078407AA
:100B8000BA0720F0621B730B840BBA0BEE1F88F7B9
:100B9000E095089598D088F09F5790F0B92F992745
:100BA000B751A0F0D1F0660F771F881F991F1AF078
:100BB000BA95C9F712C0B13081F09FD0B1E0089565
:100BC0009CC0672F782F8827B85F39F0B93FCCF3E6
:100BD000869577956795B395D9F73EF4909580956E
:100BE000709561957F4F8F4F9F4F0895E89409C08E
:100BF00097FB3EF490958095709561957F4F8F4F50
:100C00009F4F9923A9F0F92F96E9BB279395F69565
:100C1000879577956795B795F111F8CFFAF4BB0FE3
:100C200011F460FF1BC06F5F7F4F8F4F9F4F16C047
:100C3000882311F096E911C0772321F09EE8872FD1
:100C4000762F05C0662371F096E8862F70E060E08D
:100C50002AF09A95660F771F881FDAF7880F969506
:100C6000879597F9089597F99F6780E870E060E0AD
:100C700008959FEF80EC089500240A941616170635
:100C800018060906089500240A941216130614067D
:100C900005060895092E0394000C11F4882352F0E0
:100CA000BB0F40F4BF2B11F460FF04C06F5F7F4F98
:100CB0008F4F9F4F089557FD9058440F551F59F07F
:100CC0005F3F71F04795880F97FB991F61F09F3F39
:100CD00079F087950895121613061406551FF2CF62
:100CE0004695F1DF08C0161617061806991FF1CFB2
:100CF00086957105610508940895E894BB276627D9
:100D00007727CB0197F908950BD0C4CFB5DF28F032
:100D1000BADF18F0952309F0A6CFABCF1124EECFA0
:100D2000CADFA0F3959FD1F3950F50E0551F629F46
:100D3000F001729FBB27F00DB11D639FAA27F00D34
:100D4000B11DAA1F649F6627B00DA11D661F829F5B
:100D50002227B00DA11D621F739FB00DA11D621F40
:100D6000839FA00D611D221F749F3327A00D611D5D
:100D7000231F849F600D211D822F762F6A2F11243F
:100D80009F5750408AF0E1F088234AF0EE0FFF1F92
:100D9000BB1F661F771F881F91505040A9F79E3FC9
:100DA000510570F060CFAACF5F3FECF3983EDCF3C3
:100DB000869577956795B795F795E7959F5FC1F706
:100DC000FE2B880F911D9695879597F90895A3E1BD
:100DD000B0E0EDEEF6E00C94620A7C011B016A01C2
:100DE000FC0117821682838181FF66C3BE016F5F9B
:100DF0007F4F4B01F7019381F10193FD859193FFA3
:100E000081911F01882309F453C3853239F493FD7E
:100E1000859193FF81911F01853239F4B70190E0EC
:100E20000E94870B56016501E5CF10E0512C20E0B0
:100E30002032A0F48B3269F030F4803259F08332E2
:100E400069F420612CC08D3239F0803339F421608F
:100E500026C02260246023C0286021C027FD27C04F
:100E600030ED380F3A3078F426FF06C0FAE01F9FC5
:100E7000300D1124132F13C06AE0569E300D11243B
:100E8000532E20620CC08E3221F426FD11C3206443
:100E900006C08C3611F4206802C0883641F4F10196
:100EA00093FD859193FF81911F018111C1CF9BEB30
:100EB000980F933018F42061805E06C09BE9980F6C
:100EC000933008F0AAC12F7E26FF16E02F73722EF2
:100ED000853621F4F22FF0647F2E08C0863621F487
:100EE000622F6068762E02C01111115077FE07C084
:100EF0001C3348F444244394410E27E00BC01830BF
:100F000030F4212F06C027E04CE3442E03C027E035
:100F100017E0412C560174E0A70EB11CF601608168
:100F2000718182819381042DA4010E94990A6C0130
:100F3000098100FF02C003FF06C071FC07C072FCFC
:100F400008C0612C08C03DE2632E05C02BE2622E72
:100F500002C090E2692E802F8C7099F1662011F00A
:100F600084E001C083E0851510F0512C0BC0581AA5
:100F700073FC08C0B70180E290E00E94870B5A948E
:100F8000C9F7F3CF662029F0B701862D90E00E94C3
:100F9000870B03FD03C000E810E002C00CE710E07F
:100FA000F72DF0717F2EF8018491882309F476C221
:100FB00071108052B70190E00E94870B0F5F1F4FA6
:100FC000F2CF77FE0FC04C0C04FF04C08A8181333E
:100FD00009F44A94141474F5F8E0F41578F588E0EF
:100FE000482E2CC076FC2AC0812F90E08C159D05E0
:100FF0009CF06CEFC6166FEFD60674F0772D706814
:10100000772E0AC0E2E0F0E0EC0FFD1FE10FF11DCA
:101010008081803319F411501111F4CF77FE0EC086
:1010200044244394410E812F90E0C816D9062CF435
:101030001C1904C04424439401C010E077FE07C08B
:101040001C141D043CF496012F5F3F4F05C025E0A2
:1010500030E002C021E030E0662011F02F5F3F4F0A
:10106000112331F0412F50E04F5F5F4F240F351FA8
:10107000452D50E02417350714F4521A01C0512CA5
:10108000872D897049F4552039F0B70180E290E04E
:101090000E94870B5A94F7CF662029F0B701862D5E
:1010A00090E00E94870B73FC09C0552039F0B7010E
:1010B00080E390E00E94870B5A94F7CF77FE5FC0E1
:1010C0009C2D8D2DD7FE02C090E080E0692E782EF9
:1010D00040E050E0C601841991099D878C879601F4
:1010E00026193709280D391D812F90E0EE27FF279B
:1010F000E81BF90BFF87EE87FFEF6F167F0669F499
:10110000B7018EE290E02B8B3A8B488B598B0E9473
:10111000870B598948893A892B89C614D70454F01A
:101120006C857D85661577052CF4F901E40FF51FB4
:10113000818101C080E371E0671A71084F5F5F4FE2
:10114000EE85FF856E167F066CF0B70190E02B8B65
:101150003A8B488B598B0E94870B2B893A89488997
:101160005989CACF6C147D0439F49A81963318F4E6
:10117000953311F404FF81E3B70190E04BC08A81FD
:10118000813309F00F7EB70190E00E94870B1111A7
:1011900005C074FE18C085E490E017C0B7018EE268
:1011A00090E00E94870B82E066246394680EF4014D
:1011B000E80FF11D8081B70190E00E94870B11506C
:1011C00041F3862DF1CF85E690E0B7010E94870BB1
:1011D000D7FC05C0C114D10439F404FF05C0D19473
:1011E000C194D1088DE201C08BE2B70190E00E946A
:1011F000870B80E36AE0C616D1042CF08F5FFAE01B
:10120000CF1AD108F7CFB70190E00E94870BB70142
:10121000C601C0960E94870B41C1833631F08337E7
:1012200079F0833509F058C021C0560172E0A70E4D
:10123000B11CF6018081898301E010E0640114C0D3
:101240005601F2E0AF0EB11CF601C080D18026FF3E
:1012500003C0612F70E002C06FEF7FEFC6012B8BE0
:101260000E947C0B8C012B892F7715C05601F2E070
:10127000AF0EB11CF601C080D18026FF03C0612FE4
:1012800070E002C06FEF7FEFC6012B8B0E94710BE5
:101290008C012B892068722E23FD1AC0852D90E0C9
:1012A00008171907A8F4B70180E290E00E94870BA5
:1012B0005A94F4CFF60177FC859177FE81916F0106
:1012C000B70190E00E94870B51105A940150110908
:1012D0000115110579F7E2C0843611F0893651F510
:1012E000560127FF09C0F4E0AF0EB11CF601608182
:1012F0007181828193810AC0F2E0AF0EB11CF601C8
:1013000060817181882777FD8095982F022F0F7655
:1013100097FF08C090958095709561957F4F8F4F8E
:101320009F4F00682AE030E0A4010E941A0CC82EEA
:10133000C8183EC0022F853721F40F7E2AE030E026
:101340001DC0097F8F3691F018F4883559F0B0C070
:10135000803719F0883711F0ABC0006104FF09C075
:10136000046007C024FF08C0066006C028E030E023
:1013700005C020E130E002C020E132E0560107FF65
:1013800009C0F4E0AF0EB11CF60160817181828169
:10139000938108C0F2E0AF0EB11CF601608171814B
:1013A00080E090E0A4010E941A0CC82EC8180F77A4
:1013B00006FF0BC0202F2E7FC11650F404FF0AC079
:1013C00002FD08C0202F2E7E05C0DC2C202F03C07C
:1013D000DC2C01C0D12E24FF0DC0FE01EC0DF11D4F
:1013E0008081803311F4297E09C022FF06C0D39486
:1013F000D39404C0822F867809F0D39423FD13C0C0
:1014000020FF06C01C2DD51418F4150D1D19D52C60
:10141000D51468F4B70180E290E02B8B0E94870B13
:10142000D3942B89F5CFD51410F45D1801C0512C3D
:1014300024FF12C0B70180E390E02B8B0E94870B42
:101440002B8922FF17C021FF03C088E590E002C06E
:1014500088E790E0B7010CC0822F867859F021FD13
:1014600002C080E201C08BE227FD8DE2B70190E06F
:101470000E94870BC11638F4B70180E390E00E9408
:10148000870B1150F7CFCA94F401EC0DF11D808148
:10149000B70190E00E94870BC110F5CF552009F4E9
:1014A000C2CCB70180E290E00E94870B5A94F6CF3D
:1014B000F7018681978102C08FEF9FEF6396E2E18B
:1014C0000C947E0A2F923F924F925F926F927F927E
:1014D0008F929F92AF92BF92CF92DF92EF92FF9244
:1014E0000F931F93CF93DF93CDB7DEB7CA1BDB0BF0
:1014F0000FB6F894DEBF0FBECDBF09942A88398895
:1015000048885F846E847D848C849B84AA84B9849B
:10151000C884DF80EE80FD800C811B81AA81B981A7
:10152000CE0FD11D0FB6F894DEBF0FBECDBFED01BB
:101530000895283008F027E03327DA01990F311D8C
:1015400087FD916000966105710539F432602E5F68
:101550003D9330E32A95E1F708959F3F30F08038BE
:101560007105610509F03C5F3C5F3D93913008F0E7
:101570008068911DDF93CF931F930F93FF92EF929B
:10158000192F987F9695E92F96959695E90FFF2745
:10159000E252FF4F99273327EE24FF24A701E701EA
:1015A00005900894079428F4360FE71EF81E491F8B
:1015B000511D660F771F881F991F0694A1F705908C
:1015C000079428F4E70EF81E491F561FC11D770F18
:1015D000881F991F661F0694A1F70590079428F4A9
:1015E000F80E491F561FC71FD11D880F991F661F70
:1015F000771F0694A1F70590079420F4490F561F12
:10160000C71FD81F990F661F771F881F0694A9F759
:1016100084911095177041F0D695C79557954795C9
:10162000F794E7941A95C1F7E4E8F0E06894159010
:10163000159135916591959105907FE27395E1182B
:10164000F10A430B560BC90BD009C0F7E10CF11E90
:10165000431F561FC91FD01D7EF4703311F48A95A5
:10166000E6CFE894015030F0080F0AF40027021783
:1016700008F4202F2395022F7A3328F079E37D9305
:101680002A95E9F710C07D932A9589F606949795D7
:101690006795379517951794E118F10A430B560B88
:1016A000C90BD00998F023957E9173957A3308F091
:1016B00070E37C932013B8F77E9170617D9330F0D6
:1016C000839571E37D9370E32A95E1F71124EF9000
:1016D000FF900F911F91CF91DF91992787FD9095F2
:1016E0000895FC010590615070400110D8F7809575
:1016F00090958E0F9F1F0895FC01615070400190DE
:101700000110D8F7809590958E0F9F1F08950F9325
:101710001F93CF93DF93182F092FEB018B8181FD4E
:1017200003C08FEF9FEF20C082FF10C04E815F810A
:101730002C813D81421753077CF4E881F9819F0198
:101740002F5F3F4F39832883108306C0E885F985D2
:10175000812F0995892B29F72E813F812F5F3F4FDC
:101760003F832E83812F902FDF91CF911F910F9177
:101770000895A0E0B0E0EFEBFBE00C94680A6B0189
:101780004A017901D90113962C9121FF1DC0C0E0B7
:10179000D0E0C815D905D9F08C015C01AC0CBD1C9A
:1017A000C8010A151B0571F00F5F1F4FD70118966E
:1017B000ED91FC911997B701DC018C910995892B6A
:1017C00079F305C02196E5CF80E090E001C0CE011D
:1017D000CDB7DEB7ECE00C94840A0F931F93CF9340
:1017E000DF93E091D601F091D701238121FF1BC047
:1017F000EC0100E010E089916091D6017091D70171
:10180000DB011896ED91FC911997882331F0099529
:10181000892B89F30FEF1FEFEECF8AE00995892B13
:1018200011F4C80102C08FEF9FEFDF91CF911F919C
:101830000F910895FA01AA27283051F1203181F142
:10184000E8946F936E7F6E5F7F4F8F4F9F4FAF4FC8
:10185000B1E03ED0B4E03CD0670F781F891F9A1FDB
:10186000A11D680F791F8A1F911DA11D6A0F711D8F
:10187000811D911DA11D20D009F468943F912AE09B
:10188000269F11243019305D3193DEF6CF01089583
:10189000462F4770405D4193B3E00FD0C9F7F6CFB4
:1018A000462F4F70405D4A3318F0495D31FD40527C
:1018B000419302D0A9F7EACFB4E0A6959795879512
:1018C00077956795BA95C9F70097610571050895F1
:1018D0009B01AC010A2E069457954795379527959D
:1018E000BA95C9F7620F731F841F951FA01D089535
:0418F000F894FFCF9A
:1018F4000000000200000000FE00000000000000E4
:10190400000200000000DE000000000048454C4CCE
:101914004F0D00FFFFFFFFFFFFFFFFFFFFFFFFFF74
:10192400FFFFFF0020204F56455243555252454E6B
:04193400542020001B
:00000001FF
